S31508001800080A0020D9180008E7180008E91800088F
S3150800181000000000000000000000000000000000BA
S315080018200000000000000000000000000119000888
S3150800183000000000000000000319000841360008F7
S31508001840E5440008071900080719000807190008E1
S31508001850071900080719000807190008B92500081C
S315080018600719000855230008071900080719000872
S31508001870071900080719000807190008AD380008F5
S3150800188001390008000000000000000007190008E0
S3150800189000000000071900080719000807190008C2
S315080018A0000000000719000807190008853C000811
S315080018B007190008071900080719000800000000A2
S315080018C0EE11AA550348854600F024FA0048004759
S315080018D0595E0008080A00200B4880F308880B4860
S315080018E080470B480047FEE704207146084202D0AD
S315080018F0EFF3098001E0EFF30880714604F090F8F1
S31508001900FEE7FEE7FEE7FEE7080A00204138000882
S31508001910C518000830B50B460146002020220124D0
S3150800192009E00D46D5409D4205D31D469540491B05
S315080019302546954040191546521E002DF1DC30BD4E
S3150800194070B500242546002801DA01244042002902
S3150800195001DA01254942FFF7DDFFAC4200D04042DB
S31508001960002C00D0494270BD03460B439B0703D0A9
S3150800197009E008C9121F08C0042AFAD203E00B7846
S315080019800370401C491C521EF9D27047D2B201E0BE
S315080019900270401C491EFBD270470022F6E710B5BC
S315080019A013460A4604461946FFF7F0FF204610BDBF
S315080019B0F8B502464A40D40F42004B0052085B086D
S315080019C09A4202D20246084611464A0023D0C30D5F
S315080019D04A00DDB2120EAD1A202D35DA490201266B
S315080019E0490AF6058A19002C00D0524220214F1BBD
S315080019F01146B9402A411018C20D9A4221D0002C2E
S31508001A0017D0012D08DCDA05801AD20F8019D20703
S31508001A10DBB200F045F9F8BDDA05801A012340006B
S31508001A201B06C01880185A428018CA0F104349006E
S31508001A3007E04908C2071143DA05801A80194008E9
S31508001A40801800F025F9F8BD61000122511A001B23
S31508001A50F7E70122D2075140AAE70122D2075040F0
S31508001A60A6E7024670B54A40D30FDB0740002DD0E3
S31508001A704A002AD0010E140E000212020919400A61
S31508001A80520A8418E50104465443000A120A2E0431
S31508001A905043A4194219200CC543AA18120C012553
S31508001AA0AD03521C521912047F39240400D0521C6B
S31508001AB0104301D44000491EC2B20C06C0092018C2
S31508001AC0401C4008802A02D003E0002070BD400870
S31508001AD04000002900DA0020184370BD70B50246A0
S31508001AE04A40D50F40004A00ED0740085208002832
S31508001AF014D0002A12D0C40DD30D41020120C0050E
S31508001B005202490A520AE41A091812187D349142F7
S31508001B1001D3641C00E04900002C01DA002070BDE6
S31508001B200023914201D3891A03434008490000283B
S31508001B30F7D100290AD0914202D10121C90705E04F
S31508001B40914201D2012101E00121C943E005C018F3
S31508001B50401900F09DF870BD10B500229623114675
S31508001B6000F09EF810BD410040020122400AD2054D
S31508001B70090E80187F2901DA00207047962903DCB0
S31508001B809622511AC8407047963988407047C20F46
S31508001B90D207400040080BD0C10D0723DB01C91846
S31508001BA040020905400A1143C2084007114370471D
S31508001BB0002001467047000010B5002904DB012407
S31508001BC0E40740428C412146002B04DB1C460123D6
S31508001BD0DB075242A3418B4200D1824210BD00006E
S31508001BE010B5002904DB0124E40740428C41214654
S31508001BF0002B04DB1C460123DB075242A341994212
S31508001C0000D1904210BD00000122D207002800DB57
S31508001C10101A002900DB511A814270470122D207A7
S31508001C20002800DB101A002900DB511A8842704789
S31508001C30F0B51FB40646002082B00546402401913F
S31508001C4000901BE0019922460F46304600F084F8C2
S31508001C50049A059B801A994110D3104619462246C4
S31508001C6000F06AF8361A8F410197224601200021B2
S31508001C70009F00F061F838184D4100902046641E18
S31508001C800028DFDC019B00982946324607B0F0BDE4
S31508001C90002904DA401C490001D140084000704779
S31508001CA070B40024050C05D11024000402D10029C3
S31508001CB021D01124050E01D100020834050F01D1E7
S31508001CC00001241D850F01D18000A41C002801DB1A
S31508001CD04000641C002908D020252E1B0D46F5401F
S31508001CE0A14000D001212943084301061B1B000A15
S31508001CF0DB1D02D5002070BC7047DB05181880185C
S31508001D000029F8DA401C4900F5D170BC40084000AB
S31508001D1070470000064C0125064E05E0E36807CC2F
S31508001D202B430C3C98471034B442F7D3FFF7CEFD4B
S31508001D30786B0008986B000810B5202A04DB01466A
S31508001D40203A9140002010BD914020239C1A03465A
S31508001D50E3401943904010BD10B5202A04DB08461D
S31508001D60203AD040002110BD0B46D340D040202455
S31508001D70A21A91400843194610BD000010B5044642
S31508001D80002C08D101210920C00600F0B5FE00206C
S31508001D9000F0AAF852E0012C05D102210920C0065C
S31508001DA000F0AAFE4AE0022C05D104210920C0064B
S31508001DB000F0A2FE42E0032C05D108210920C00646
S31508001DC000F09AFE3AE0042C05D110210920C0063D
S31508001DD000F092FE32E0052C05D120210920C0062C
S31508001DE000F08AFE2AE0062C05D140210920C0060B
S31508001DF000F082FE22E0072C05D180210920C006CA
S31508001E0000F07AFE1AE0082C04D101210D4800F0F2
S31508001E1073FE13E0092C04D102210A4800F06CFE77
S31508001E200CE00B2C04D11021064800F065FE05E0F5
S31508001E300C2C03D18021034800F05EFE204600F0FA
S31508001E4053F810BD000400487FB5002000900190AB
S31508001E500290039000241BE000250CE0E8000E49E0
S31508001E6040186100405AA1006A4651584018A1001E
S31508001E705050681C85B2142DF0DBA1006A465058F4
S31508001E801421FFF747FD6100044A5052601C84B2D2
S31508001E90042CE1DB7FBD0000600400204C0100201B
S31508001EA000B587B001A800F0AFF80121480201F09B
S31508001EB039FA002001903020029001204002039058
S31508001EC000200690059001A9064800F031F8012186
S31508001ED0044800F021F80121024800F011F807B083
S31508001EE000BD00000024014010B504460723002267
S31508001EF02146024800F038F810BD000000240140D1
S31508001F00002904D0426801231A43426003E042686C
S31508001F105208520042607047002904D0826808239C
S31508001F201A43826003E0826808239A4382607047F6
S31508001F3042680B4B1A4042600B684A681A4343686A
S31508001F401A4342608268074B1A4082600B694A69E5
S31508001F501A438B681A4383681A43826070470000E5
S31508001F600FBCFFFF8FF1F9FFF0B504460D46164684
S31508001F701F463F073F0F2B46082B0FD91B071B0F82
S31508001F80083B606F9A000F21914088436067606F35
S31508001F9099003A468A40104360670BE0206F9A0022
S31508001FA00F21914088432067206F99003A468A405E
S31508001FB010432067E0680121A9408843E060E06893
S31508001FC00121A9400843E060012080032840002839
S31508001FD003D0012000F020F807E00120C0032840C4
S31508001FE0002802D0012000F017F8F0BD002905D01E
S31508001FF08268FF2301331A43826004E08268FF2364
S3150800200001339A4382607047002101604160816014
S315080020100173016141617047002806D00649496885
S315080020200C221143044A516005E0034949680C2211
S315080020309143014A516070470024014010B5074892
S315080020400078002806D0FFF7FFFE00200349087035
S3150800205000F09CFD7E2002F051FA10BD54010020CC
S31508002060FFB583B00C46029400200190002726E0B5
S3150800207000261CE0721C039951430846791CFFF799
S3150800208049FC0546A54201D9281B00E0601B054608
S315080020900298A84204D90295059806700698077012
S315080020A00298002802D10120019002E0761C402EF9
S315080020B0E0D300BF0198002800D002E07F1C042F5F
S315080020C0D6D300BF029807B0F0BD000000BF00BF1E
S315080020D000BF00BF00BFBFF34F8F00BF00BF00BFE8
S315080020E006480749C86000BF00BF00BFBFF34F8F4F
S315080020F000BF00BF00BF00BF00BFFDE70400FA0530
S3150800210000ED00E010B500F001F810BD10B5234849
S315080021100078002817D1224801F08CF901283CD113
S315080021201F480078002838DD1D480078402834DC30
S3150800213001F07BFD1B490860012018490870002042
S315080021401949087029E0164A17490978491C501890
S3150800215001F070F9012816D113480078401C12497D
S3150800216008700F4800780978884216D100200B4974
S3150800217008700B484078FF280FD10B4800780228D2
S315080021800BD1FFF7A3FF01F050FD0649096864313A
S31508002190884202D900200149087010BD210100209B
S315080021A0E4030020240100202001002078B502461F
S315080021B0002327E0002020E08400155B441CA400CF
S315080021C0145BA54218DD8400A5182E886C46268067
S315080021D06D8865808400A518441CA400A418268868
S315080021E02E8064886C80441CA400A5186C4624883C
S315080021F02C806C4664886C80401C4C1EE41A844211
S31508002200DADC5B1C4C1E9C42D4DC78BD10B586B06B
S3150800221004460121880301F085F80121880401F0AC
S3150800222061F803221146224800F051FC03220421DA
S315080022301F4800F04CFC01A801F0C9FD01943021AB
S315080022406846018100214181818101821821C1816D
S3150800225001A9184801F078FD0121164801F051FD41
S3150800226005A800F08AFC082168468182012181754B
S315080022701821C17505A90E4800F0DCFB1021684637
S3150800228081824821C17505A9094800F0D3FB1B21A5
S3150800229068460170032141700121817000F088FFB2
S315080022A001220221034801F044FD06B010BD0000DA
S315080022B0000400480038014070B502460B46FF2569
S315080022C0FF2408E01178521C69400748405C6040CA
S315080022D005460648445C18465E1EB3B20028F1D18E
S315080022E02802204370BD000078690008786A000853
S315080022F001B506490098086002E07E2002F0FEF863
S31508002300024800680028F8D108BD00002C0100200A
S31508002310014600220E4B1A61CA005A6100229A61D0
S3150800232005221A6100BF0A4A1069C207D20F002A9D
S3150800233004D0012212040240002AF4D0044A126989
S3150800234052085200024B1A6100229A617047000037
S3150800235000E000E010B500210848FFF747FE02201C
S3150800236000F052F801200649087001020920C0064B
S3150800237000F0FFFB02F0EAFA10BD0000002401405D
S315080023805C01002000B589B00121084600F0AAFFCB
S315080023901A4800F045F801A800F08EF81848019090
S315080023A01848029000216846017304200490684684
S315080023B00175802141754900C18289000183202168
S315080023C08176090281830021C183018401A90B4812
S315080023D000F04CF80121094800F01CF801220221FE
S315080023E0064800F039F80921684601700221417053
S315080023F00121817000F0DCFE09B000BD0800024032
S315080024000024014028040020014948607047000064
S31508002410000002400268520852000A4302607047F0
S3150800242010B504462068400840002060002020605F
S315080024306060A060E060E1B2084608380521FFF751
S3150800244069FA01460F20884002494968084301494C
S31508002450486010BD00000240002A03D003680B4301
S31508002460036002E003688B430360704710B50A7A7D
S315080024708B7D1A430B7C1A434B7C1A434B8A1A43AF
S315080024808B8A1A430B8B1A434B8B1A430368094CE6
S3150800249023401A43026002680123DB039A438B8BAD
S315080024A01A430260CA6842600A6882604A68C26063
S315080024B010BD00000F80FFFF00210160416001721E
S315080024C0C1600174417441828182817501834183AF
S315080024D08183704770B506460C4621460A4800F0C7
S315080024E00FFA0546002D01D1401E70BD06488542EB
S315080024F002D10648051B00E02D1B22462946304618
S31508002500FFF732FA2046F0E700F4000800FC00085E
S3150800251070B506460C4621460A4800F0F1F905460C
S31508002520002D01D1401E70BD0648854202D10648DD
S31508002530051B00E02D1B224629463046FFF714FAF4
S315080025402046F0E700F0000800F8000870B50646D7
S315080025500C4621460A4800F0D3F90546002D01D15C
S31508002560401E70BD0648854202D10648051B00E09C
S315080025702D1B224629463046FFF7F6F92046F0E796
S3150800258000F800080000010870B505460C4622460A
S315080025900249284600F075F9204670BD00F4000887
S315080025A070B505460C4622460249284600F069F9E8
S315080025B0204670BD00F0000810B5024800F004F887
S315080025C010BD0000208000000149486170470000E6
S315080025D0000401401CB5684600F0A9F80F21002048
S315080025E000F07CF80120C0030090002168460171C4
S315080025F0102141710121817100F010F80521002098
S3150800260000F06CF820200090002168460171102126
S3150800261041710121817100F001F81CBD8179002901
S3150800262048D02D490968026891432B4A1160114622
S31508002630496802689143284A51600179002906D100
S315080026401146096802681143234A116005E02249C8
S31508002650496802681143204A51601F49896802681F
S3150800266091431D4A91601146C968026891431A4A06
S31508002670D160417910290CD1114689680268114345
S31508002680154A91601146C96802681143124AD16019
S3150800269020E04179082906D10F4989680268114363
S315080026A00D4A916016E00C49C968026811430A4A46
S315080026B0D1600FE00179002906D107490968026847
S315080026C09143054A116005E0034949680268914348
S315080026D0014A5160704700000004014010B50D4AD8
S315080026E08B109B00D3588A07140F0F22A2409343DE
S315080026F0084A8C10A40013518B109B00D2588B07E4
S315080027001C0F0346A3401A43024B8C10A4001A510F
S3150800271010BD00000800014008B507216846017091
S31508002720022141700121817000F042FD08BD00219F
S31508002730016001710C21417100218171704700000F
S3150800274010B504460848006902210843064908618D
S315080027500846446100694021084303490861034863
S3150800276000F00EF910BD000000200240FF0F000027
S315080027700C48C068C007C00F002801D00120704768
S315080027800848C06804210840002801D00220F6E75E
S315080027900448C06810210840002801D00320EEE74D
S315080027A00420ECE700200240034800698021084322
S315080027B001490861704700000020024030B5044610
S315080027C00D4605480069012108430349086125802B
S315080027D00F2000F0D5F830BD0020024010B57E204D
S315080027E001F08CFE064800F00FF87E2001F086FE08
S315080027F0044800F009F87E2001F080FE10BD0000B4
S3150800280000F4000800F0000810B5044600F0ACF823
S315080028102046FFF795FFFFF7C7FF10BD70B50346C3
S315080028200125002208E050001C5A0748844201D0BE
S31508002830002506E0501C82B2CE0F76187610964216
S31508002840F1DC00BF284670BDFFFF0000F8B505465D
S315080028500E46144600F088F87E2001F04FFE002749
S3150800286007E029883046FFF7A9FFB61CAD1C781C7F
S3150800287087B2E10F09194910B942F2DCFFF794FF54
S31508002880F8BDF8B507460C4615462946204600F019
S3150800289037F80646002E0DD12046FFF7B5FF012072
S315080028A080022018FFF7B0FF2A4621463846FFF770
S315080028B0CDFF24E0012080022018401BB0420AD137
S315080028C0012080022018FFF79FFF2A463146384626
S315080028D0FFF7BCFF13E00120C0022018401BB042DE
S315080028E008D12046FFF790FF2A4631463846FFF7BB
S315080028F0ADFF04E02A4631463846FFF7A7FFF8BD84
S31508002900F8B505460E462F46E807C00F002801D041
S3150800291000BFFEE731460120C002FFF711F8002983
S3150800292001D000BFFEE700240BE02046704347199C
S3150800293031463846FFF772FF012800D108E0601CCF
S3150800294084B231460120C002FEF7FAFFA042ECDC51
S3150800295000BF31460120C002FEF7F2FFA04200D1B7
S3150800296000273846F8BD0000024803494860034876
S31508002970486070472301674500200240AB89EFCDC8
S3150800298010B5024600BFFFF7F3FE0346521EFF24AA
S3150800299000E0641E002CFCD1012B01D1002AF2D1E3
S315080029A00648006977218843044908613420C860CD
S315080029B0002A01D1052010BD1846FCE70020024078
S315080029C008B5684600F0D9F801210F20400400F048
S315080029D089FC0021C943684601800021C170694607
S315080029E00920C00600F026F80021C9436846018080
S315080029F00021C17069460C4800F01CF80021C94343
S31508002A00684601800021C1706946084800F012F83E
S31508002A100021C943684601800021C17069460448FF
S31508002A2000F008F808BD0000000400480008004847
S31508002A30000C0048F8B50246CD782F073F0FCD7831
S31508002A4010263540002D01D08D782F4314460020DE
S31508002A5011E085062B0E0D88012686403540002D8F
S31508002A6007D025680F269E40B5433E469E4035430F
S31508002A702560451CE8B20828EBDB141D0D882D12CD
S31508002A800095002011E085062B0E01258540009E45
S31508002A903540002D07D025680F269E40B5433E4693
S31508002AA09E4035432560451CE8B20828EBDBCD7807
S31508002AB0282D04D155690E883543556106E0CD7831
S31508002AC0482D03D115690E8835431561F8BD70B5D3
S31508002AD04D07EB0E082902DA0546203501E00546C2
S31508002AE024352C460F269E402568B54316469E403B
S31508002AF03543256070BD000038B504460D460920EB
S31508002B00C006844203D10121480400F0EBFB1148BA
S31508002B10844203D10121000200F0E4FB0E488442FE
S31508002B2003D10121000200F0DDFB0C48844203D1E9
S31508002B300121080500F0D6FB684600F01EF8684635
S31508002B400580012181700021C17069462046FFF782
S31508002B5071FF38BD0004004800080048000C004812
S31508002B60024690680840002801D0012070470020DE
S31508002B70FCE741617047016170470021C943018044
S31508002B80022181700421C17070470000F0B587B03A
S31508002B90002006900590049003907E2001F0AEFC7C
S31508002BA0002611E07100B64A505AFEF7D5FF0546D1
S31508002BB0B449FEF793FF0446B349FEF752FFB10046
S31508002BC0B24A5050701C86B2042EEBDBAF4A5168ED
S31508002BD09068FEF73EFF0446AD49FEF77FFF069074
S31508002BE0AA4948680699FEF779FFAA490860AA48DB
S31508002BF0807B00283FD1A84910318889FEF7ACFFB1
S31508002C00A54910310190C888FEF7A6FFA349009090
S31508002C10FEF764FF07460199FEF723FF0546A0491C
S31508002C20FEF75CFF04469C4910318889FEF794FF3D
S31508002C3007469B49FEF752FF05469648016828460F
S31508002C40FEF70BFF21460290FEF748FF04909249D3
S31508002C5010314889FEF780FF05460499FEF7A8FE5D
S31508002C600446FEF780FF8F4908600846008881B24F
S31508002C708D48818134E08C48007D002830D1864813
S31508002C80C078012829D183480068FEF780FF0446EA
S31508002C90864A874BFEF7A4FF1CD27E480068FEF7DB
S31508002CA076FF0446834A844BFEF786FF12D27C4998
S31508002CB078480068FEF7D5FE0446FEF754FF81B251
S31508002CC07548103081810146888903F017FA02F0A9
S31508002CD097FD02E0022003F075FA00216E48817321
S31508002CE06D48C07B012804D102F08AFD00216A489C
S31508002CF0C1736D498889FEF72FFF704908606349DB
S31508002D0008686F49FEF7ADFE054601218907FEF7FB
S31508002D10A8FE0446FEF727FF81B263484181FF38C3
S31508002D20C1380088FF21F531884272DD00205A49F2
S31508002D30343908805848C07801283ED15A48007D61
S31508002D4000283AD0514988685D49FEF78AFE04464C
S31508002D50FEF709FF85B24D4948685949FEF781FED5
S31508002D600446FEF700FF80B2854210D14A4834383F
S31508002D70C068AF218900884209D94B4840790028A4
S31508002D8005D145493439C8600421474841713F494E
S31508002D9088680021FEF738FF05D03C4948680021BD
S31508002DA0FEF732FF09D140484079002805D13A4953
S31508002DB03439C86005213C4841713449C868FEF772
S31508002DC0E6FE04463F4A404BFEF7F6FE22D22F495E
S31508002DD0C868FEF7DCFE04463C4A3D4BFEF7ECFEAF
S31508002DE013D220213B48FFF7BBFE00280DD12E4801
S31508002DF00079012809D12C484079002805D12649AF
S31508002E003439C86006212848417101212248417099
S31508002E1011E033E01D49C8682F49FEF7FFFE0AD2C4
S31508002E202148007D002803D100211B48417002E09B
S31508002E300121194841701549C8682849FEF7EEFE70
S31508002E4003D201211448017102E0002112480171E0
S31508002E501148407800280DD113480079012804D17B
S31508002E6004211C48FFF785FE08E004211948FFF7EE
S31508002E7082FE03E004211748FFF77DFE07B0F0BD88
S31508002E804C01002000F07F450000A04050040020BF
S31508002E903333A34060010020000200200024744957
S31508002EA000007A44680100208C0300206666666686
S31508002EB06666E63FCDCCCCCCCCCCEC3FA403002058
S31508002EC00000C842A245B6F3FDD4EC3F759318043A
S31508002ED0560EDD3F0004004852B89E3FFCA97940D3
S31508002EE00148006870470000300100200348006868
S31508002EF003490978401801490860704730010020E5
S31508002F003801002008B50121480400F0EBF9012139
S31508002F10880400F0E7F96846FFF72FFE04216846A3
S31508002F2001804821C17069460920C006FFF782FD65
S31508002F306846FFF722FEFF210131684601804821D5
S31508002F40C17069460748FFF775FD6846FFF715FE25
S31508002F502021684601800421C17069460148FFF7AF
S31508002F6069FD08BD0004004810B504210920C00603
S31508002F70FFF7F6FD00286FD15E48407A00285FD13A
S31508002F805C48007901283DD15A48007D002839D18E
S31508002F9059480078401C58490870084600780428A3
S31508002FA023DB56A001F0FAFA00205349087051486D
S31508002FB07C38408900280AD152485349C860012103
S31508002FC051483430C172FF30113041810AE0022184
S31508002FD04D483430C17200204B49C860002145482D
S31508002FE07C38418101F0AAFA0CE0434800780228AF
S31508002FF008DC4548C0687D210901884202D90020BD
S315080030004149C8603B48007D002816D13E48C06942
S315080030103E49884211D337487C384089002805D173
S315080030203B483949C8610020C86006E03248007844
S31508003030022802DC00203449C86001212D4841726B
S315080030403448007800280ED1012032490870012141
S315080030502848017207E0FFE700202E490870002182
S31508003060244801724172284800697D21C9008842B6
S315080030703AD929A001F092FA0020234908610021D3
S315080030801C480172007D002828D11A487C384088DF
S31508003090032829DA17487C384089002824D11A4899
S315080030A03430007900280ED11248007901281BD146
S315080030B001211048017500201349C86001211248F2
S315080030C03430C17210E00B48407900280CD1012138
S315080030D00848417100200C49C86005E000200A49EB
S315080030E0C8600021034801717E2001F007FA0148F3
S315080030F0007A10BD8C030020760100204C4F434B0C
S3150800310045442100DC050000CC0100203075000094
S31508003110606D0000770100200A53746172742057AD
S315080031206F726B0A000000001CB50121480400F00C
S31508003130D9F80121880400F0D5F801A8FFF71DFD8C
S31508003140442168468180012181711021C17101A93C
S315080031501548FFF76FFC1549684681800121817182
S315080031601021C17101A90920C006FFF763FC0821D7
S315080031700920C006FFF7FFFC00BF802168460180D2
S315080031800021C17069460920C006FFF753FC2021BB
S315080031900920C006FFF7EFFC00BF10210920C00672
S315080031A0FFF7E9FC1CBD0000000400487981000017
S315080031B08178002925D01749032212028918027836
S315080031C092109200895802789207D30EFF229A40ED
S315080031D0914342789207120E03789B07DB0E9A40BA
S315080031E011430C4A03231B02D21803789B109B0039
S315080031F0D1500178CA06D20E01219140054A1160C4
S3150800320007E00178CA06D20E01219140014A8032B0
S315080032101160704700E100E009480A49486000204B
S3150800322048875A2088870887074808630020C862A5
S3150800323006484862064888620448C8617047000024
S3150800324000003443A40300209A99993E00002041C7
S31508003250000048420D4A12689208920002430B4B3E
S315080032601A600B4A126904231A43094B1A61012989
S3150800327001D130BF02E040BF20BF20BF044A126917
S3150800328004239A43024B1A617047000000700040FD
S3150800329000ED00E010B501F001F940210F48FFF7F5
S315080032A068FC40210920C006FFF763FC00210C4892
S315080032B0FEF726FE00210A48FEF72EFEFFF780FBE2
S315080032C001F0ECF80121080700F01CF80121084676
S315080032D0FFF7C0FF00F0B4FA10BD00000004004874
S315080032E000240140002905D0054A52690243044BCF
S315080032F05A6104E0024A52698243014B5A61704797
S3150800330000100240002905D0054AD2690243044B41
S31508003310DA6104E0024AD2698243014BDA617047F6
S3150800332000100240002905D0054A92690243044B61
S315080033309A6104E0024A92698243014B9A61704796
S315080033400010024010B500F031F804494968F0222F
S3150800335011400909024A515CC84010BD00100240DC
S31508003360FC00002010B5FFF7EDFF05494968072264
S3150800337012021140090A034A515CC84010BD0000F8
S3150800338000100240FC00002010B5FFF7DBFF0549DE
S3150800339049680722D2021140C90A034A515CC8404B
S315080033A010BD000000100240FC000020F8B51E48C1
S315080033B040680C210840042802D008282ED101E0D4
S315080033C01A4C2DE0184840300069C007C00F002885
S315080033D00AD015484030006902210840002801D06B
S315080033E0134802E0114800E0104807460E484030EE
S315080033F00069FF2109040840000C451C0A484030B2
S315080034000069072109020840000A461C3946694333
S3150800341008463146FEF77EFA044601E0034C00BF33
S3150800342000BF2046F8BD00000010024000127A00D6
S3150800343000093D0070B5044600250221074800F042
S3150800344066FC002808D0054800F0BAFC2070022166
S31508003450024800F054FC0125284670BD003801409A
S3150800346010B500F001F810BD00B585B062480068D7
S31508003470012108436049086000BF5F4800680221CF
S3150800348008400028F9D05D485D4908605D48006835
S31508003490102108435B49086008460068C008C00058
S315080034A0086057490968481E5749FEF733FA0490D9
S315080034B05448006804994907490F08435149086068
S315080034C04D484068514908404B494860084640689D
S315080034D0902108434849486008464068486048487B
S315080034E000684649884207D94348406805210902C9
S315080034F00843414948600BE041480068444988420E
S3150800350006D93D4840680121890208433A4948607E
S315080035106B4601AA3A4801683E48FEF7A1FD3648BF
S315080035204030006980088000334940310861084608
S315080035300069400840000861684600784007400F67
S315080035400290684600794006400E03902A48C069F2
S31508003550890508432849C8612748403000692E492B
S315080035600840254940310861039800040299090278
S31508003570084321494031096908431F494031086118
S315080035801D4800680121090608431B49086000E038
S3150800359000BF194800680121490608400028F7D0ED
S315080035A01548406880088000134948600846406806
S315080035B0022108431049486000E000BF0E484068F1
S315080035C00C2108400828F8D10120FEF7A1FE0A4878
S315080035D0406810218843084948600120FEF798FE94
S315080035E00548406880218843034948600120FEF762
S315080035F08FFE05B000BD00000010024000A24A047C
S315080036000C0100200020024000366E010FC0FFFFAB
S315080036100051250200127A00FFF800FF042806D19F
S315080036200649096904221143044A116105E0034960
S31508003630096904229143014A1161704700E000E0DC
S3150800364010B5FFF753FC75480088401C734908807D
S315080036500846C068401CC86071480088401C70490C
S31508003660088070480068002804D06E480068401E2C
S315080036706C4908606C48007A012805D167480069DA
S31508003680401C6649086102E00020644908616348F5
S315080036903430007A01280ED160484069401C5F49E1
S315080036A04861084640696149884207D900215B4854
S315080036B03430017202E000205849486157483430D6
S315080036C0807A012805D15548C06A401C5349C8620A
S315080036D002E000205149C8625348007D002809D0FD
S315080036E04E484068401C4D4948600846806A401C60
S315080036F0886203E000204949486088624A48807920
S3150800370004280AD14548C0694949884208D243482D
S31508003710C069401C4149C86102E000203F49C861B0
S31508003720FF2101314348FFF71BFA002813D03B4815
S315080037303430407800280ED13B48007901280AD158
S315080037403648006A3949884208D23448006A401C1B
S315080037503249086202E00020304908622F483430B6
S31508003760C07A012813D1C1030920C006FFF703FA5E
S315080037702A4881688068401C284A9060FF20F530F6
S31508003780814225D9002110463430C17220E02348F1
S315080037903430C07A022812D181030920C006FFF707
S315080037A0EAF91E4881688068401C1C4A90602248D5
S315080037B081420DD9002110463430C17208E000203C
S315080037C0164988600121C9030920C006FFF7D1F907
S315080037D01548007D012805D11048006B401C0F498B
S315080037E0086302E000200D4908637E2000F086FE8B
S315080037F020211048FFF7B4F900280AD00748406A84
S315080038000E49884208D20548406A401C0349486266
S3150800381002E000200149486210BD0000CC010020EA
S31508003820280100202C0100208C03002088130000AA
S3150800383050C3000000040048DC050000B8880000FA
S3150800384010B516480068012108431449086008465F
S3150800385040681349084011494860084600681149FC
S3150800386008400E4908600846006801218904884313
S315080038700A49086008464068C3210904884307497D
S3150800388048600846006808490840044908609F20BF
S3150800389000048860FFF7E4FD10BD00000010024038
S315080038A00CC0FFF8FFFFF6FEFFFF8F0010B50421DE
S315080038B0080700F017F9002806D00421080700F0C9
S315080038C0EBF801210148817010BD000000020020BC
S315080038D008B501214804FFF705FD02220121092048
S315080038E0C006FFF7F4F80221684601801821C17066
S315080038F00121817069460920C006FFF79BF808BDBB
S3150800390010B50121164800F0EDF8002827D001214E
S31508003910134800F0C1F81348807801281FD11248CF
S31508003920C179C079401CC2B20F48C2710B2916DD95
S315080039300C48C078012804D101020920C006FFF707
S315080039401AF90948C0790D2809DD00210548817052
S3150800395001210648FEF74AFB00210348C17110BD44
S3150800396000040040000200208C03002000240140CF
S3150800397030B589B004460D4601210846FFF7C2FC5A
S3150800398006A800F049F907946846058300210184D2
S3150800399008A881706846817606A90120800700F08C
S315080039A005F90F216846017101214171817101A84C
S315080039B0FFF7FEFB0421080700F06AF8012204213C
S315080039C0080700F09CF802A800F0DCF860216846B9
S315080039D0017201214172002003900021684601749A
S315080039E002A90120800700F095F80821C80600F012
S315080039F0C1F84021080600F06DF80121880700F09B
S31508003A003BF80121880700F057F80121880700F0E4
S31508003A1047F809B030BD00007FB504460D460121C0
S31508003A200220FFF76FFC684600F0F6F80194684636
S31508003A300580002101818172817069460D4800F078
S31508003A40B5F810216846017302214173012181737B
S31508003A5003A8FFF7ADFB0121064800F019F801227B
S31508003A601146044800F04BF80121024800F018F806
S31508003A707FBD000000040040002904D002688023AE
S31508003A801A43026003E0026880239A430260704783
S31508003A9002698A430261704702698A430261704774
S31508003AA0002904D0026801231A43026003E0026871
S31508003AB05208520002607047002905D0426C012363
S31508003AC0DB031A43426404E0426C0123DB039A4396
S31508003AD042647047826907231B039A430B021A4301
S31508003AE082617047024610690840002805D0D068F0
S31508003AF00840002801D0012070470020FCE7002A72
S31508003B0003D0C3680B43C36002E0C3688B43C3603A
S31508003B107047000010B5826907231B039A430B7888
S31508003B201B021A4382610A7A12014B781B011A4357
S31508003B30036A3024A3431A4302624A6882630C4A22
S31508003B40904213D14A7A12018B781B011A43036AF1
S31508003B50C024A3431A4302624A8992008B899B00B8
S31508003B601A4343682401A3431A43426010BD000068
S31508003B70002C014082690123DB029A430B021A4397
S31508003B808261704700210170417081704160017245
S31508003B90417241818181704701229207904201D189
S31508003BA0816301E08AB282637047000002680323DA
S31508003BB01B029A430B891A430260134A904206D0A5
S31508003BC001229207904202D0104A904205D102681B
S31508003BD070239A438B781A4302600B4A904205D0A9
S31508003BE00B4A904202D00B4A904205D1026B120A48
S31508003BF012028B7A1A4302634A68C2620A88826290
S31508003C000122426170470000002C01400004004078
S31508003C1000440140004801400021C9434160002199
S31508003C200180018181708172704710B5FFF758F9DC
S31508003C3010BD000070B5FFF785FB05467D21C9005C
S31508003C40FDF768FE0446601E0C49884200D90CE060
S31508003C50601E0B4948610321081F00F0BDFC0020C7
S31508003C60074988610720086100BF0420FFF7D6FCD2
S31508003C700021481E00F0B0FC70BD0000FFFFFF00E9
S31508003C8000E000E010B502210A4800F049F80028D3
S31508003C900ED0084800F094F8C4B20748407A0028C5
S31508003CA002D1204601F0FAFD0221024800F027F869
S31508003CB010BD0000003801400002002010B504467F
S31508003CC02146054800F080F800BF0121024800F0AF
S31508003CD01EF80028F9D010BD0038014070B504461A
S31508003CE00D467E2000F00AFC03E02078641CFFF7EE
S31508003CF0E5FF2846691E8DB20028F6D170BD4161E0
S31508003D0070478269520852000A4382617047024628
S31508003D1090680840002801D0012070470020FCE781
S31508003D200246D0680840002801D0012070470020CC
S31508003D30FCE7002A03D003690B43036102E0036929
S31508003D408B4303617047000070B504460D46002694
S31508003D50E0693021884329790843E061E069442114
S31508003D608843A9790843E061E06980088000297AD8
S31508003D700843E061A0691821884369890843A0615E
S31508003D80A06904218843297B0843A0610B48844223
S31508003D9003D1FFF7F9FA064602E0FFF7E3FA06460B
S31508003DA030462968FDF7B6FD0009206230462968C5
S31508003DB0FDF7B0FD0007000F606270BD00380140D6
S31508003DC001464868C0B27047CAB2026070474B21C4
S31508003DD0C901016030210171002181710172182128
S31508003DE0418100210173704710B51D4840880300C2
S31508003DF000F0E4FB0504111E2B2C2D0018487C301E
S31508003E004089FF218A31884204DC01211448418017
S31508003E1000F094FB1BE012487C304089FF216F318B
S31508003E20884204DC02210E48418000F087FB0EE040
S31508003E300B487C304089FF215531884204DC032138
S31508003E400748418000F07AFB01E000E000BF00BFB0
S31508003E5003487C300079002801D100F06FFB10BDC3
S31508003E601003002008B59E484088002806D001287F
S31508003E706ED002287ED0032869D1DFE00221984857
S31508003E807C30817120219748FEF76AFE002841D0D0
S31508003E909549C868FF21F531FDF73CFDC007C00FFD
S31508003EA000281CD110210920C006FEF762FE082151
S31508003EB00920C006FEF75DFE00BF20216846018086
S31508003EC0012181701021C17069460920C006FEF7DC
S31508003ED0B1FD20210920C006FEF74BFE37E0102170
S31508003EE00920C006FEF747FE08210920C006FEF78E
S31508003EF042FE00BF8021684601800021C1706946E4
S31508003F000920C006FEF796FD20210920C006FEF707
S31508003F1032FE1CE010210920C006FEF72AFE082101
S31508003F200920C006FEF725FE00BF2021684601804D
S31508003F30012181701021C17069460920C006FEF76B
S31508003F4079FD20210920C006FEF713FE00BFC5E053
S31508003F50012163487C30817120216248FEF700FE0A
S31508003F60002817D06049C868FF21F531FDF7D2FC53
S31508003F70C00700E02AE0C00F002805D10821092063
S31508003F80C006FEF7F6FD0AE008210920C006FEF77E
S31508003F90F2FD04E008210920C006FEF7EAFD10211B
S31508003FA00920C006FEF7E7FD00BF802168460180AC
S31508003FB00021C17069460920C006FEF73BFD202195
S31508003FC00920C006FEF7D7FD00BF87E02021454837
S31508003FD0FEF7C6FD002815D04349C868FF21F5310C
S31508003FE0FDF798FCC007C00F002805D1102109204D
S31508003FF0C006FEF7C0FD0AE010210920C006FEF73C
S31508004000B8FD04E010210920C006FEF7B2FD08211C
S315080040100920C006FEF7AFFD00BF80216846018073
S315080040200021C17069460920C006FEF703FD20215C
S315080040300920C006FEF79FFD00BF4FE02021294852
S31508004040FEF78EFD002815D02749C868FF21F531EF
S31508004050FDF760FCC007C00F002805D11021092014
S31508004060C006FEF788FD22E010210920C006FEF7EB
S3150800407080FD1CE01C49C868CD21FDF74BFCC00734
S31508004080C00F002805D110210920C006FEF773FDD0
S315080040900DE01549C868CD21FDF73CFCC007C00FE7
S315080040A0002804D010210920C006FEF762FD082169
S315080040B00920C006FEF75FFD00BF80216846018023
S315080040C00021C17069460920C006FEF7B3FC20210D
S315080040D00920C006FEF74FFD00BF00BF00BF08BDA0
S315080040E01003002000040048CC01002008B5042174
S315080040F0E54881718079030000F060FA050451985B
S31508004100FEFDFC00E0484089FF218A31884203DB36
S315080041100121DD48817141E0DB484089FF21873173
S3150800412088420ADDD8487C384088022805D0022112
S31508004130D5487C38418000F001FA2021D348FEF7A3
S315080041400FFD00282AD0D249C868FF21F531FDF7AE
S31508004150E1FBC007C00F002805D110210920C006C1
S31508004160FEF709FD04E010210920C006FEF701FD4F
S3150800417000BF8021684601800021C1706946092078
S31508004180C006FEF757FC20210920C006FEF7F3FCFF
S3150800419000BF08210920C006FEF7EDFC72E1BA4807
S315080041A04089FF21A231884203DB0221B64881718A
S315080041B03BE02021B548FEF7D3FC002835D0B449AA
S315080041C0C868FF21F531FDF7A5FBC007C00F002819
S315080041D005D108210920C006FEF7CDFC04E0082118
S315080041E00920C006FEF7C5FC10210920C006FEF707
S315080041F0C2FC00BF8021684601800021C170694663
S315080042000920C006FEF716FC20210920C006FEF785
S31508004210B2FC00BF9C487C384088012805D00121A3
S3150800422099487C38418000F089F92BE19648408905
S31508004230FF21A531884203DB03219348817165E09C
S3150800424020219248FEF78CFC00285FD0FF2101311F
S315080042508E48FEF785FC002807D08D48006A8D49F0
S31508004260884202D90421884881718949C868FF2192
S31508004270F531FDF74FFBC007C00F00281CD11021F0
S315080042800920C006FEF775FC08210920C006FEF7BE
S3150800429070FC00BF20216846018001218170102131
S315080042A0C17069460920C006FEF7C4FB2021092013
S315080042B0C006FEF75EFC1AE010210920C006FEF7CC
S315080042C05AFC00BF8021684601800021C1706946FA
S315080042D00920C006FEF7AEFB20210920C006FEF71E
S315080042E04AFC00BF08210920C006FEF744FC6648C0
S315080042F07C3802E0C5E06DE009E04088002805D07A
S31508004300002161487C38418000F018F9BAE0202184
S315080043105E48FEF725FC00285BD0FF2101315B488B
S31508004320FEF71EFC002807D05948006A59498842FA
S3150800433002D90421544881715549C868FF21F531CD
S31508004340FDF7E8FAC007C00F00281CD11021092084
S31508004350C006FEF70EFC08210920C006FEF709FC78
S3150800436000BF202168460180012181701021C1709B
S3150800437069460920C006FEF75DFB20210920C00614
S31508004380FEF7F7FB1AE010210920C006FEF7F3FB3B
S3150800439000BF8021684601800021C1706946092056
S315080043A0C006FEF747FB20210920C006FEF7E3FBFF
S315080043B000BF08210920C006FEF7DDFB32487C381D
S315080043C04088002805D000212F487C38418000F01D
S315080043D0B5F857E020212D48FEF7C2FB00284FD03C
S315080043E029487C384088002805D0002126487C3892
S315080043F0418000F0A3F82648C069274988421CD2A4
S3150800440010210920C006FEF7B4FB08210920C006C2
S31508004410FEF7AFFB00BF20216846018001218170AD
S315080044201021C17069460920C006FEF703FB20214A
S315080044300920C006FEF79DFB1AE010210920C006D8
S31508004440FEF799FB00BF8021684601800021C170F4
S3150800445069460920C006FEF7EDFA20210920C006A4
S31508004460FEF789FB00BF08210920C006FEF783FB7B
S31508004470074834304078012802D103210248817167
S3150800448000E000BF00BF08BD8C0300200004004800
S31508004490CC010020941100003075000010B5FEF71D
S315080044A03BF9FEF797F802F037F810BD0348806825
S315080044B0400840000149886070470000002C004011
S315080044C080210143014A116070470000002C00401A
S315080044D003488068002801D0012070470020FCE7C7
S315080044E0002C004010B5FFF7F3FF002804D0FFF7B3
S315080044F0DDFF662000F002F810BD00004106490EF7
S31508004500014A116070470000002C004004494968C0
S31508004510FF22813291430143014A516070470000EE
S31508004520002C004004494968C909C9014206520ECF
S315080045301143014A51607047002C004010B57E2097
S31508004540FFF7DCFF0948FEF75FF90949094881804A
S315080045500621001D00F03AFA0649091D8881402205
S3150800456002490448001DFEF78CF910BD00F8000842
S31508004570FBAA00000C03002070B505460C46012175
S31508004580C802FEF7BFFEFF208130FFF7BFFF2046B7
S31508004590FFF7C8FF2846FFF793FF70BD0FB410B5A5
S315080045A003A9044B044A029800F062F810BC08BC40
S315080045B004B0184779580008C801002030B474467A
S315080045C0641E2578641CAB4204D3635D5B00E31864
S315080045D030BC18471D46F8E710B5002819DB1A4AFB
S315080045E003231B02D21883089B00D2588307DC0ECC
S315080045F0FF23A3409A438B071B0E8407E40EA340B0
S315080046001A43114B032424021B198408A4001A51C7
S3150800461018E00E4A03071B0F083B9B089B00D2585D
S315080046208307DC0EFF23A3409A438B071B0E8407E0
S31508004630E40EA3401A43054B0407240F083CA408BC
S31508004640A4001A5110BD000000E100E01CED00E0D6
S3150800465002E008C8121F08C1002AFAD1704770473D
S31508004660002001E001C1121F002AFBD1704700009B
S31508004670FFB58FB00F460446002606E025280AD067
S31508004680129A11999047641C761C20780028F5D157
S31508004690304613B0F0BD00250121A14A009500E07F
S315080046A00543641C23780846203B98401042F7D1FE
S315080046B020782E2815D1042005436078641C2A2802
S315080046C00AD101CF641C00900BE000990A225143DD
S315080046D030394018641C0090207801463039092981
S315080046E0F3D920786C280ED004DC4C2813D06A281D
S315080046F012D104E074280ED07A280DD10BE00120DF
S315080047004005054307E00121090562780D43824209
S3150800471001D16D18641C641C2078864669284AD025
S3150800472008DC0028B4D058286DD0632810D0642837
S3150800473008D140E070286BD0732812D0752860D055
S31508004740782860D0129A704611999047761CE5E051
S315080047503878694608720020487202A8019001203C
S3150800476003E0386801900020C0433F1D69070CD557
S31508004770002500E06D1C00998D420FDA8542F9DBB1
S315080047800199495D0029F5D108E0002500E06D1C76
S315080047908542FCDB0199495D0029F8D1761907E0C5
S315080047A0019801990078491C0191129A119990472C
S315080047B06D1EF5D2B2E00A20029000216802400F71
S315080047C0039102280CD001CFC117844600290DDABF
S315080047D06246084652420021814194462D2008E04F
S315080047E0FF1DFF08FF0003CF8446EFE7280504D521
S315080047F02B206A46107401203CE0E8073AD02020B6
S31508004800F7E70A2000E0102000210391029007E054
S3150800481010200290002104200543082003910090EF
S315080048206802400F022810D001CF002184460020DC
S315080048300D9028071FD5704670280CD0029A1020B4
S31508004840039B42401A430CD015E0FF1DFF08FF00EA
S3150800485003CF8446EBE740206A46107401200D908A
S315080048600CE06046084306D030206A46107470464D
S31508004870507402200D907046582804D029A0019043
S315080048800DA80E900DE02CA0F9E76046039B029A4E
S31508004890FDF7CEF9019B84469B5C0E9A521E0E923A
S315080048A0137060460843F0D10E9805A9081A2030FF
S315080048B00190680701D5009801E001200090019950
S315080048C0884203DD01460198081A00E00020002509
S315080048D0009006E004A8129A405D119990476D1C55
S315080048E0761C0D988542F5DB04E0129A3020119962
S315080048F09047761C0099481E00900029F5DC08E0D0
S315080049000E980E990078491C0E91129A11999047A3
S31508004910761C0199481E01900029F1DC641CB4E656
S315080049200928010030313233343536373839616277
S31508004930636465660000000030313233343536373B
S3150800494038394142434445460000000010B519482D
S31508004950007801282DD100201649087016490880CC
S3150800496012E01548008840001449085A1449098875
S31508004970C900144A8918104A1288520088520E48EB
S315080049800088401C0C4908800B4800880428E8DB8E
S315080049907E20FFF7B3FD0A480088401C08490880B6
S315080049A008460088142804DB0020088001200649F0
S315080049B0087010BD5C010020720100202804002048
S315080049C074010020600400205401002010B502463E
S315080049D00023002901D1002010BD03E01488921C91
S315080049E0E01883B208464C1EA1B20028F6D1184634
S315080049F0F2E7000010B5FEF723FFFEF783FAFEF78D
S31508004A0093FBFDF7BFFCFDF74BFA0B20FDF7B6F954
S31508004A100C20FDF7B3F90320FDF7B0F90420FDF7E4
S31508004A20ADF901212048FDF7E1FAE1204002FDF742
S31508004A30EDFB01211D480171002101754171FF3807
S31508004A408D3841718171012118484172FEF78CFA3F
S31508004A50FEF73EFF16496320FEF78AFF1A216320F8
S31508004A60FEF7DAFFFFF7E6F810487C384089002899
S31508004A7001D1FFF7F7F97F217E20FFF77DFD0021A1
S31508004A800C48417040210920C006FEF774F8402101
S31508004A900948FEF770F8FFF701FD0020074908707E
S31508004AA004493439C86010BD002401408C03002035
S31508004AB0581B000000020020000400487601002070
S31508004AC070B50025A748807A01280ED1A548343844
S31508004AD0C06AFF21F531884207D90021A1488172B1
S31508004AE00020A1490880A14908709E48407A0128FB
S31508004AF070D19D48007A012811D003280ED19C4810
S31508004B00007D002806D19748007A002802D10121A5
S31508004B109448017200209349343948611BE1924850
S31508004B20407A07286FD007DC0300FFF747FD071216
S31508004B3023568583959683000A2879D004DC0828AD
S31508004B4077D0092876D1B0E0A12874D0A528F9D164
S31508004B50FBE0002083493439486101218148C1714D
S31508004B60002202218348FFF7E4F800207D49343902
S31508004B70C860EEE000207B49343948617A48807A7B
S31508004B80012811D17848007B282825DA7648007B49
S31508004B900A2821DD7448017B7248103041810121C1
S31508004BA010388173C17017E06F48807A022812D1D5
S31508004BB06D4A117BD07A00F027FF0546282D0BDABF
S31508004BC00A2D09DD674810304581012110388173A7
S31508004BD0C17001E0C3E070BDBBE000206149343913
S31508004BE048616148807A022821D15F4A117BD07AD0
S31508004BF000F00AFF012807D103215D4801755EA070
S31508004C00FFF7CCFC13E038E0574A117BD07A00F066
S31508004C10FBFE00280BD10021554801755148C07B81
S31508004C20012804D100F0ECFD00214E48C17390E044
S31508004C3082E032E08CE085E04B48807A02280AD18F
S31508004C40494A117BD07A00F0DFFE46491031C88008
S31508004C5001214448C1737CE07BE000204149343996
S31508004C604861414A117BD07A00F0CEFE3D491031A9
S31508004C704880012001F0A6FA6BE000203949343952
S31508004C804861394A117BD07A00F0BEFE35491031A9
S31508004C908880032001F096FA5BE000203149343918
S31508004CA04861022001F08EFA53E000202D4934397C
S31508004CB048612D49887AC117890F09188910890012
S31508004CC0411A33D12849887AC117890F09188910DA
S31508004CD0244A10321181104600891C2826DA00243D
S31508004CE01FE0A200921D204B9B1D995CA200521D3D
S31508004CF0985C00F089FE0146A2001A481E308152CF
S31508004D00A2000832184B9B1D995CA200D21D985C24
S31508004D1000F07AFE0146A20012481E3010184180A3
S31508004D20641C104810300089A042DADC042001F027
S31508004D3049FA00F065FD0CE0052001F043FA00F0A1
S31508004D405FFD06E001F006FA03E001F09FF900E0D6
S31508004D5000BF00BF00BF00BF00210248417200BF6C
S31508004D6039E700000002002000050020C5010020E8
S31508004D708C030020003801400A484F545F310A006E
S31508004D8070B505460C46002D02D0012D1ED10CE04B
S31508004D90602101208007FEF79DFE00210120800783
S31508004DA0FEF7FAFE0A48047010E009480078A042A7
S31508004DB009D0602101208007FEF78CFE21460120DC
S31508004DC08007FEF7E9FE0248047000BF00BF70BD09
S31508004DD07801002008B5FE480079012879D1FD48F8
S31508004DE0007D0028FAD1FA4840790300FFF7E6FB70
S31508004DF008050772D8F1F0EFEEED002008BDF54979
S31508004E002039C868FF219131FCF784FD8007800F9F
S31508004E1000280AD110210920C006FDF7ACFE08219A
S31508004E200920C006FDF7A7FE40E0EA492039C86810
S31508004E30FF219131FCF76EFD8007800F01280AD10A
S31508004E4010210920C006FDF794FE08210920C00696
S31508004E50FDF791FE2AE0DF492039C868FF21913124
S31508004E60FCF758FD8007800F02280AD11021092077
S31508004E70C006FDF780FE08210920C006FDF77BFE67
S31508004E8014E0D4492039C868FF219131FCF742FD66
S31508004E908007800F032809D108210920C006FDF7DD
S31508004EA068FE10210920C006FDF765FE00BF8021B7
S31508004EB0684601800021C17069460920C006FDF7D1
S31508004EC0B9FD20210920C006FDF755FE00BF0120C7
S31508004ED094E7E2E1BF492039C868C821FCF71AFD02
S31508004EE08007800F00280AD110210920C006FDF787
S31508004EF042FE08210920C006FDF73DFE3DE0B54902
S31508004F002039C868C821FCF705FD8007800F0128ED
S31508004F100AD110210920C006FDF72BFE0821092019
S31508004F20C006FDF728FE28E0AA492039C868C82126
S31508004F30FCF7F0FC8007800F02280AD1102109200F
S31508004F40C006FDF718FE08210920C006FDF713FE66
S31508004F5013E0A0492039C868C821FCF7DBFC8007A4
S31508004F60800F032809D108210920C006FDF701FE94
S31508004F7010210920C006FDF7FEFD00BF8021684606
S31508004F8001800021C17069460920C006FDF752FD5F
S31508004F9020210920C006FDF7EEFD00BF01202DE700
S31508004FA08C492039C868C821FCF7B4FC8007800FF3
S31508004FB000280FD110210920C006FDF7DCFD0821C5
S31508004FC00920C006FDF7D7FD42E065E12FE1C4E000
S31508004FD08AE050E07F492039C868C821FCF79AFC66
S31508004FE08007800F01280AD110210920C006FDF785
S31508004FF0C0FD08210920C006FDF7BDFD28E075495A
S315080050002039C868C821FCF785FC8007800F02286C
S315080050100AD110210920C006FDF7ADFD0821092097
S31508005020C006FDF7A8FD13E06A492039C868C821FB
S31508005030FCF770FC8007800F032809D10821092096
S31508005040C006FDF796FD10210920C006FDF793FD61
S3150800505000BF8021684601800021C1706946092089
S31508005060C006FDF7E7FC20210920C006FDF783FDF1
S3150800507000BF0120C2E657492039C868FF212D31F3
S31508005080FCF748FCC007C00F002805D110210920ED
S31508005090C006FDF770FD0FE04E492039C868FF21AC
S315080050A02D31FCF737FCC007C00F002804D01021AB
S315080050B00920C006FDF75DFD00BF80216846018016
S315080050C00021C17069460920C006FDF7B3FC2021FE
S315080050D00920C006FDF74FFD00BF08210920C006BC
S315080050E0FDF749FD012089E63A492039C868FF21BC
S315080050F09131FCF70FFCC007C00F002805D110211D
S315080051000920C006FDF737FD0FE032492039C86887
S31508005110FF219131FCF7FEFBC007C00F002804D021
S3150800512010210920C006FDF724FD00BF802168462E
S3150800513001800021C17069460920C006FDF77AFC86
S3150800514020210920C006FDF716FD00BF0821092009
S31508005150C006FDF710FD012050E61E492039C86833
S31508005160C821FCF7D7FB8007800F00280AD1102139
S315080051700920C006FDF7FFFC08210920C006FDF737
S31508005180FAFC41E013492039C868C821FCF7C2FB7C
S315080051908007800F01280AD110210920C006FDF7D3
S315080051A0E8FC08210920C006FDF7E5FC2CE00949C2
S315080051B02039C868C821FCF7ADFB8007800F022894
S315080051C00FD110210920C006FDF7D5FC082103E000
S315080051D08C030020EC0100200920C006FDF7CBFC5B
S315080051E012E02F49C868C821FCF794FB8007800F96
S315080051F0032809D108210920C006FDF7BAFC1021A9
S315080052000920C006FDF7B7FC00BF8021684601806B
S315080052100021C17069460920C006FDF70BFC202154
S315080052200920C006FDF7A7FC00BF0120E6E51C49DA
S31508005230C868C821FCF76EFBC007C00F002805D157
S3150800524010210920C006FDF796FC0DE01449C86830
S31508005250C821FCF75FFBC007C00F002804D0102147
S315080052600920C006FDF785FC00BF8021684601803D
S315080052700021C17069460920C006FDF7DBFB202125
S315080052800920C006FDF777FC00BF08210920C006E3
S31508005290FDF771FC0120B1E500BF00BFAEE50000D7
S315080052A0CC01002008B5FC48007D002838D0FB4812
S315080052B0C078012834D1F9483438C068F84988429A
S315080052C00ED9F548808964280ADAF3484079002817
S315080052D006D10721F04841710020F0493439C860E9
S315080052E0ED48007D03281BD0EB488089FF21EB3170
S315080052F0884215DDE8488189EAA0FFF74FF9E648B4
S31508005300407900280CD1E5483438C068EA49884213
S3150800531006D90321E04841710020E0493439C860C4
S31508005320DD48007901287DD1DB4840790300FFF785
S3150800533045F90805074E97DDFEFDFCFB002008BD74
S31508005340D6483438C068E121C900884239D90821CD
S315080053500920C006FDF70FFC00BF802168460180C2
S315080053600021C17069460920C006FDF763FB2021AC
S315080053700920C006FDF7FFFB00BF10210920C00663
S31508005380FDF7F9FB0121C5481438017514308079F9
S31508005390002807D1C1493439C8600021BE480171C7
S315080053A041710AE0BD483438C068AF210901884216
S315080053B003D90020B9493439C8600121B748417179
S315080053C003E00021B548143801750120B7E7B34852
S315080053D03438C068B94988423CD908210920C00632
S315080053E0FDF7C9FB00BF8021684601800021C17016
S315080053F069460920C006FDF71DFB20210920C006C5
S31508005400FDF7B9FB00BF10210920C006FDF7B3FB65
S315080054100121A248143801751430807900280DD16D
S315080054209E4900E09CE13439C86000219A48017120
S315080054304171002099493439C8600FE097483438DB
S31508005440C068AF210901884208D900209349343938
S31508005450C86003E0002191481438017501206EE701
S315080054608E483438C0689649884239D908210920B7
S31508005470C006FDF780FB00BF802168460180002139
S31508005480C17069460920C006FDF7D4FA2021092013
S31508005490C006FDF770FB00BF10210920C006FDF706
S315080054A06AFB01217D48143801751430807900287B
S315080054B00BD17A493439C8600021774801714171A6
S315080054C0002076493439C8600EE074483438C0681C
S315080054D07C49884208D9002070493439C86003E0FD
S315080054E000216E4814380175012028E76B483438C6
S315080054F0C0687D21090188423ED908210920C006D5
S31508005500FDF739FB00BF8021684601800021C17084
S3150800551069460920C006FDF78DFA20210920C00634
S31508005520FDF729FB00BF03E019E1D4E072E029E0AA
S3150800553010210920C006FDF71EFB01215748143823
S3150800554001751430807900280BD154493439C86064
S315080055500021514801714171002050493439C86011
S315080055600EE04E483438C0685349884208D90020AE
S315080055704A493439C86003E000214848143801759F
S315080055800120DCE645483438C068E121C900884274
S315080055903AD908210920C006FDF7EDFA00BF802197
S315080055A0684601800021C17069460920C006FDF7DA
S315080055B041FA20210920C006FDF7DDFA00BF1021B7
S315080055C00920C006FDF7D7FA0121344814380175B9
S315080055D01430807900280BD130493439C86000214D
S315080055E02D480171417100202C493439C8600FE0FB
S315080055F02A483438C068AF210901884208D90020F2
S3150800560026493439C86003E0002124481438017556
S31508005610012094E621483438C0682A49C8398842A6
S3150800562054D908210920C006FDF7A5FA00BF802134
S31508005630684601800021C17069460920C006FDF749
S31508005640F9F920210920C006FDF795FA00BF1021B7
S315080056500920C006FDF78FFA012110481438017594
S315080056601430807900280BD10C493439C8600021E0
S31508005670094801714171002008493439C86028E099
S3150800568006483438C0681049884222D900200349A0
S315080056903439C8601DE000008C0300200002002099
S315080056A0204E00000A675F776F726B2E74656D7007
S315080056B05F313A25640A0000B80B0000A406000012
S315080056C0C4090000AC0D0000CC10000000212548DC
S315080056D00175012033E623482038C06822498842EC
S315080056E038D908210920C006FDF745FA00BF8021F0
S315080056F0684601800021C17069460920C006FDF789
S3150800570099F920210920C006FDF735FA00BF1021B6
S315080057100920C006FDF72FFA012112480175143039
S31508005720807900280BD10F492039C86000210F481D
S315080057300171417100200B492039C8600DE0094804
S315080057402038C0680A49884207D900200549203907
S31508005750C86002E00021034801750120EFE500BF9B
S3150800576000BFECE5EC010020A40600008C03002035
S315080057708C0A000010B5052416E0FF2101311F48E8
S31508005780FCF70BF9FF2101311C48FCF7A3FEFE21AB
S315080057901A48FCF791FD01461848C030C08F81426F
S315080057A002D100F055FC10BD2046611ECCB200287F
S315080057B0E3D1052416E0FF2101311048FCF7EDF886
S315080057C0FF2101310D48FCF7A3FEFE210B48FCF72B
S315080057D073FD01460948C030C08F814202D100F0EE
S315080057E037FCE0E72046611ECCB20028E3D100F082
S315080057F0C7F900F005F800BFD5E700001002002041
S3150800580010B5FCF7EBFF1A491A488180001D00897C
S315080058101C2815DA1748001D01890E30FCF7C6FC4E
S315080058201449091D088908E000228300114912312C
S31508005830CA52830059184A80401C1E28F4D300E037
S3150800584010BDFE210B48001DFCF736FD0146094830
S31508005850C430C187FF210131C038FCF795FEFF210E
S3150800586001310448001DFCF79BFE00BFE8E7000075
S31508005870FBAA00000C02002070B504460D46E1B2F2
S315080058800548FEF7A1FA00BF01210348FEF73FFAD3
S315080058900028F9D0204670BD0038014070B504468E
S315080058A00025012155488172002054493439C862BF
S315080058B053480088FA2804DD0020514908805149D8
S315080058C00870504800780300FEF778FE080516248D
S315080058D0384451667295AA2C0DD1012049490870A1
S315080058E0474801880088401C454A1080901D44544A
S315080058F000201146C8707FE0FB2C0AD14048018879
S315080059000088401C3E4A1080901D445402203D49A0
S31508005910087071E0012C03D103203A49087004E0AD
S31508005920032C02D1062037490870354801880088BB
S31508005930401C334A1080901D44545DE0304801886D
S315080059400088401C2E4A1080901D445404202D497E
S31508005950087051E02A48847001880088401C284A4B
S315080059601080901D445405202649087044E02448B8
S31508005970C078401CC0B22249C8708978884202DBC8
S315080059800620204908701E4801880088401C1C4AC9
S315080059901080901D44542FE0194801880088401C47
S315080059A0174A1080901D445407201649087023E0B2
S315080059B0134801880088401C114A1080901D4454E1
S315080059C0801F0188801DFCF777FC002809D100217B
S315080059D00A4881720121417200200A490870084963
S315080059E0088007480088FA2804DD00200449088052
S315080059F00449087000E000BF00BF70BD0002002027
S31508005A0000050020C501002070B502460020134697
S31508005A100C461D02FF26360235402543284670BD32
S31508005A2086B004460D4626686768A0680590E06853
S31508005A3004902069039060690290A0690190E0696A
S31508005A40009017A0FEF7AAFD31461BA0FEF7A6FD9B
S31508005A5039461CA0FEF7A2FD1DA00599FEF79EFD7E
S31508005A601EA00499FEF79AFD1FA00399FEF796FD5E
S31508005A7020A00299FEF792FD23A00199FEF78EFD5C
S31508005A8026A00099FEF78AFD2948416A29A0FEF753
S31508005A9085FD29462BA0FEF781FD00BFFEE7000025
S31508005AA05B48617264206661756C742068616E6417
S31508005AB06C65725D0D0A00005230203D2025780D78
S31508005AC00A0000005231203D2025780D0A0000000A
S31508005AD05232203D2025780D0A0000005233203D21
S31508005AE02025780D0A000000523132203D20257805
S31508005AF00D0A0000537461636B6564204C52203DA7
S31508005B002025780D0A000000537461636B656420D4
S31508005B105043203D2025780D0A0000005374616328
S31508005B206B656420505352203D2025780D0A0000ED
S31508005B3000ED00E05343425F53484353523D2578F6
S31508005B400D0A000043757272656E74204C52203D32
S31508005B502025780D0A0000000749084881800021A1
S31508005B60001D41805F21C900C180152181805F2108
S31508005B700181002141817047FBAA00000C03002027
S31508005B8000201D4A1D498A80F022091D4A801422D8
S31508005B908A8002220A8119224A81194A8A81920038
S31508005BA0CA8000BF0FE00022830014498A31CA5216
S31508005BB0830059184A80830010491231CA5283005B
S31508005BC059184A80401C1C28EDDB00220B49091D88
S31508005BD0CA81FF225F320A8214224A82FF225F327A
S31508005BE08A8200228031CA80891D4A8014228A80CE
S31508005BF0FF225F32CA807047FBAA00000C02002011
S31508005C00EE02000008B57E20FEF778FCFFF7E2F802
S31508005C10012800D108BD8C48007901287ED18A4820
S31508005C20007D002802D0012879D13FE0202187484D
S31508005C30FCF796FF00282ED18548C0698549884219
S31508005C4033D28348C0687D21090188422DD27E4817
S31508005C507C384089002802D1FEF704F925E0102196
S31508005C600920C006FCF787FF00BF8021684601802F
S31508005C700021C17069460920C006FCF7DBFE202119
S31508005C800920C006FCF777FF00BF08210920C006D7
S31508005C90FCF771FF09E06E48406A6E49884202D2F5
S31508005CA0FEF7E0F801E0FEF721FACAE06849C8689D
S31508005CB0FF21F531FBF72EFEC007C00F00281CD1C7
S31508005CC010210920C006FCF754FF08210920C00648
S31508005CD0FCF74FFF00BF2021684601800121817033
S31508005CE01021C17069460920C006FCF7A3FE2021D1
S31508005CF00920C006FCF73DFF1DE010210920C0065B
S31508005D00FCF739FF00BF8021684601800021C17079
S31508005D1069460920C006FCF78DFE01E092E00BE01B
S31508005D2020210920C006FCF726FF00BF082109200C
S31508005D30C006FCF720FF84E04348007D052842D1D1
S31508005D404349C868FF21F531FBF7E4FDC007C00FDA
S31508005D5000281CD110210920C006FCF70AFF0821DB
S31508005D600920C006FCF705FF00BF20216846018010
S31508005D70012181701021C17069460920C006FCF70F
S31508005D8059FE20210920C006FCF7F3FE58E0102131
S31508005D900920C006FCF7EFFE00BF80216846018097
S31508005DA00021C17069460920C006FCF743FE202180
S31508005DB00920C006FCF7DFFE00BF08210920C0063F
S31508005DC0FCF7D9FE3CE02048007D06281BD11021AF
S31508005DD00920C006FCF7CFFE00BF80216846018077
S31508005DE00021C17069460920C006FCF723FE202160
S31508005DF00920C006FCF7BFFE00BF08210920C0061F
S31508005E00FCF7B9FE1CE010210920C006FCF7B1FE1C
S31508005E1008210920C006FCF7ACFE00BF2021684611
S31508005E200180012181701021C17069460920C006D0
S31508005E30FCF700FE20210920C006FCF79AFE00BFE9
S31508005E4000BF00BF00BFE5E68C0300200004004841
S31508005E50CC0100203075000008B5FDF7F1FCFDF710
S31508005E6051F8FDF761F9FCF78DFAFCF719F80C20E3
S31508005E70FBF784FF0920FBF781FF0820FBF77EFF6D
S31508005E800720FBF77BFF01215748FCF7AFF8E12015
S31508005E904002FCF7BBF90121544801710021417108
S31508005EA0FF388D3841718171012150484172FDF7E3
S31508005EB05BF8FDF70DFD4E496320FDF759FD1A21E4
S31508005EC06320FDF7A9FDFFF755FCFDF7B3FE00F0CB
S31508005ED099F846487C384089002801D1FDF7C2FF69
S31508005EE000214448417040210920C006FCF743FEC2
S31508005EF040214148FCF73FFEFEF7D0FA00213D4815
S31508005F00C171FDF789F901210920C006FCF733FEA6
S31508005F1069E03848C079002802D001285ED10AE035
S31508005F20FEF7CEFDFCF78AF8FFF76CFEFDF71CF8C6
S31508005F3000F018FB56E00021084600F06FF92D48DE
S31508005F403438C0682D49884208D900212948C171CA
S31508005F50012202212A48FDF7ECFE39E025493439A9
S31508005F60C868FF21F531FBF7D5FCC007C00F00282C
S31508005F701BD110210920C006FCF7FDFD00BF8021BA
S31508005F80684601800021C17069460920C006FCF7F1
S31508005F9051FD20210920C006FCF7EDFD00BF0821B0
S31508005FA00920C006FCF7E7FD12E000BF202168467D
S31508005FB00180012181701021C17069460920C0063F
S31508005FC0FCF738FD20210920C006FCF7D2FD00BFEA
S31508005FD0FCF798F87E20FEF791FA03E000210548C1
S31508005FE0C17100BF00BF94E7002401408C03002064
S31508005FF0581B00000002002000040048204E000044
S315080060000038014010B540210F48FBF7C6FC402177
S315080060100D48FCF79BFA06210B48FEF7D7FC0A4900
S31508006020898988420AD10848001F8088074988421A
S3150800603008D0FFF791FDFEF781FA03E0FFF78CFD24
S31508006040FEF77CFA10BD000010030020FBAA000032
S3150800605010B500240C484089052803DB0A48408906
S31508006060282803DD192108484181012406480089AA
S315080060701D2803DD0124022103480181012C01D1D9
S31508006080FFF7BEFB10BD00001002002070B5A0B0DF
S315080060900025002680216846FBF77FFCAA21684672
S315080060A00170FB21417001218170A521C170124840
S315080060B0007A8006010E6846017102790E490E3192
S315080060C0401DFBF751FC68460079411D6846FCF700
S315080060D0F3F80446211268460079401D6A461154B1
S315080060E068460079801D145468460079C11D6846C3
S315080060F0FDF7F4FD20B070BD1002002030B5A1B048
S315080061000446802101A8FBF748FC0025AA21684619
S315080061100171FB214171022181710121C1710221A5
S315080061200172FF2000022040011268464172847203
S31508006130072101A8FCF7C0F80546FF200002284001
S3150800614001126846C1720573092101A8FDF7C6FD4B
S3150800615021B030BDF0B5A1B000260027802101A8E6
S31508006160FBF71BFC0025AA2168460171FB2141713A
S3150800617001218171A121C171062101720FA5027A3F
S3150800618029460930FBF7F0FB6846007A411D01A84D
S31508006190FCF792F8044621126846007A401D01AAC7
S315080061A011546846007A801D14546846007AC11D49
S315080061B001A8FDF793FD21B0F0BD00004E5F5632F1
S315080061C05F31000030B5A1B00446802101A8FBF775
S315080061D0E4FB0025AA2168460171FB2141710221D1
S315080061E081710521C17102210172FF200002204040
S315080061F00112684641728472072101A8FCF75CF80F
S315080062000546FF200002284001126846C172057340
S31508006210092101A8FDF762FD21B030BD70B504461D
S315080062200D460026002D13D10846FEF7A9FD0021CC
S31508006230AD480182FF388D3841730020AB4988622A
S31508006240AB490870A94908630021A748418249E17A
S31508006250A6483430407B00287BD1A448806AFF21B9
S31508006260F53188426ED90020A04988629E48018A85
S315080062708089814210DD9C48018A9EA0FEF78EF92E
S3150800628001219A48343041739748818901827D20DB
S31508006290C0009E4908800EE0934881892046143044
S315080062A0814208DD924800780F2804DD904800787E
S315080062B0401F8F4908708C488189204628388142BA
S315080062C034DA89487C384088002803D14820884930
S315080062D0087010E084487C384088012803D1512092
S315080062E08349087007E080487C384088022802D134
S315080062F05A207F4908707D48006B854988421ED917
S3150800630000207A4908637848418A8089814209DBF6
S3150800631075484079002805D1072173484171002046
S315080063207249C86070488189418208E070480078DF
S315080063300F2804DD6E480078001F6D4908706A480A
S31508006340818901826A4801780120FEF719FDC9E0B2
S31508006350FFE76648806A6D490988884262D9002045
S31508006360624988626048018A808981425BDA5E48B0
S31508006370818920461438814215DAFF20F5306349B1
S31508006380088059488189008A081A042805DA584875
S315080063900078801C5649087035E055480078401C3E
S315080063A0534908702FE05048818920460A388142AF
S315080063B015DAFF20F530554908804B488189008A4F
S315080063C0081A022805DA4A480078401C4849087025
S315080063D019E047480078801E4549087013E042488E
S315080063E08189601F81420EDAFF20F530474908800F
S315080063F03D488189008A081A022804DB3C4800784F
S31508006400801E3B4908703848818901828089A042EC
S3150800641054DD7D20C0003D49088035480078401E7F
S31508006420334908704AE030488089A04218DD2E4872
S315080064308089001B052809DD7D20C00033490880B6
S315080064402B480078801E2A49087034E07D20C00059
S315080064502E49088026480078401E254908702AE0FB
S3150800646021488089A04226D01F488189008A081AB7
S31508006470052805DD1E480078801C1D4908701AE0AD
S3150800648019488189601F814209DAAF2080001F49B7
S31508006490088017480078801C154908700BE01D48CD
S315080064A01A49088010488089A04204DA1048007802
S315080064B0401C0F4908700C48818901820C480078F5
S315080064C00A2803DA0A200A49087006E0084800780C
S315080064D03C2802DD3C200649087005480178012061
S315080064E0FEF74EFC70BD00008C030020CC01002096
S315080064F0F60000200A675F776F726B2E6C61737403
S315080065005F74656D703A25640A000000F800002083
S31508006510B80B0000DC05000008B501214804FCF7AB
S31508006520E1FE01218804FCF7DDFE6846FCF725FB41
S315080065300421684601804821C17069460920C006C1
S31508006540FCF778FA6846FCF718FB202168460180B4
S315080065500421C17069460248FCF76CFA08BD0000C0
S315080065600004004838B50024FEF79CFE01280CD12B
S31508006570E348C068FF21F531884205D90121C903DE
S315080065800920C006FCF7F5FA38BDDE480079002870
S3150800659075D1DD49087000210846FFF73FFE002146
S315080065A0D7483430C1701438017508210920C0064F
S315080065B0FCF7E1FA00BF8021684601800021C1701E
S315080065C069460920C006FCF735FA20210920C006CD
S315080065D0FCF7D1FA00BF10210920C006FCF7CBFA58
S315080065E00021C8480175C648C068FF21F5318842B0
S315080065F009D2C34834304079002803D10121C04864
S315080066003430C1726EE10021BD48343041713438EE
S31508006610C068BE498842F5D9BA48407A00280FD1E1
S31508006620B748C0687D214901884201D2FDF7DCFBE5
S315080066300021B44841717D204001B149C8600CE091
S31508006640B048007A012808D10020AD49C860002169
S31508006650AC4841710175012101712021AC48FCF754
S315080066607FFA002806D00021A6480175012101718C
S3150800667038E104E0FCF70EFEFEF7BCF932E1A1486A
S31508006680007D0300FDF79AFF07057797B8C1CAFE94
S31508006690760000210846FFF7C1FD99483430807B13
S315080066A0002804D1002196483430C17003E0012146
S315080066B093483430C17092483430C07B012808D1E1
S315080066C094A0FDF76BFFFFF79BF800218C48343048
S315080066D0C1738B48C068914988423CD900208A49D1
S315080066E0087087483430007A002843D1202188482A
S315080066F0FCF736FA00282AD108210920C006FCF73B
S315080067003AFA00BF8021684601800021C1706946B7
S315080067100920C006FCF78EF920210920C006FCF7DF
S315080067202AFA00BF10210920C006FCF724FAFDF753
S315080067305BFB7E20FDF7E2FE1E20FBF7D9FDFCF78A
S31508006740A9FD00206E49C860FEF754F912E0002042
S315080067506B49C8600EE06A48C068FF21F531884277
S3150800676008D968487C384089002803D10021644844
S315080067703430C172B5E0012161483430C1706049D6
S31508006780C8687D21C900FBF7C5F85D494431898889
S31508006790884206D902215B4801750121FF388D38E8
S315080067A0C1725749C86800F0BDF804460121204661
S315080067B0FFF734FD95E0012151483430C170504946
S315080067C0C86800F0AFF8044601212046FFF726FD09
S315080067D04B49C8687D21C900FBF79CF848494431F4
S315080067E049880F39884206D9012145483430C17293
S315080067F005214448017574E0012141483430C170CF
S31508006800FF204130FFF70AFD6BE001213C48343098
S31508006810C17000210846FFF701FD62E001213848F2
S315080068203430C1703438C16844304088401E7D22F7
S31508006830D2005043FF30F530814209D23049C8684A
S3150800684000F070F8044601212046FFF7E7FC2BE02C
S3150800685000210846FFF7E2FC012129483430C172BD
S315080068603438C16844304088401E7D22D2005043E7
S31508006870AF2292008018814216D300202049C860B2
S31508006880084600E011E034308079012803D106215A
S315080068901C48017502E000211A4801750121C90347
S315080068A00920C006FCF765F91BE016484079002860
S315080068B016D11348C0681A49884211D9FDF794FAC7
S315080068C000200F49C8600F487C384088032803DA3F
S315080068D001210C48017503E000210A480175017180
S315080068E000BF00BF06484068FF21F531884202D93B
S315080068F00020034948607E20FDF700FE00BF43E6FE
S31508006900CC0100208C03002076010020B80B000083
S31508006910000400487772697465000000E09304007B
S3150800692010270000F8B5054600247D21C900284631
S31508006930FAF7F0FF064600270020009000BF0BE09C
S31508006940A1000C48405AB04205DCA10009480818C5
S31508006950408800900127641C06480E380089A0422A
S31508006960EEDC002F03D103480E38008A0090009809
S31508006970F8BD00001E02002000C1814001C0804110
S3150800698001C0804100C1814001C0804100C18140F1
S3150800699000C1814001C0804101C0804100C18140E1
S315080069A000C1814001C0804100C1814001C08041D1
S315080069B001C0804100C1814001C0804100C18140C1
S315080069C000C1814001C0804100C1814001C08041B1
S315080069D001C0804100C1814000C1814001C08041A1
S315080069E001C0804100C1814001C0804100C1814091
S315080069F000C1814001C0804101C0804100C1814081
S31508006A0000C1814001C0804100C1814001C0804170
S31508006A1001C0804100C1814000C1814001C0804160
S31508006A2001C0804100C1814001C0804100C1814050
S31508006A3000C1814001C0804100C1814001C0804140
S31508006A4001C0804100C1814001C0804100C1814030
S31508006A5000C1814001C0804101C0804100C1814020
S31508006A6000C1814001C0804100C1814001C0804110
S31508006A7001C0804100C1814000C0C101C30302C2F8
S31508006A80C60607C705C5C404CC0C0DCD0FCFCE0E60
S31508006A900ACACB0BC90908C8D81819D91BDBDA1AD0
S31508006AA01EDEDF1FDD1D1CDC14D4D515D71716D640
S31508006AB0D21213D311D1D010F03031F133F3F232B0
S31508006AC036F6F737F53534F43CFCFD3DFF3F3EFE20
S31508006AD0FA3A3BFB39F9F83828E8E929EB2B2AEA90
S31508006AE0EE2E2FEF2DEDEC2CE42425E527E7E62600
S31508006AF022E2E323E12120E0A06061A163A3A26270
S31508006B0066A6A767A56564A46CACAD6DAF6F6EAEDF
S31508006B10AA6A6BAB69A9A86878B8B979BB7B7ABA4F
S31508006B20BE7E7FBF7DBDBC7CB47475B577B7B676BF
S31508006B3072B2B373B17170B050909151935352922F
S31508006B4096565797559594549C5C5D9D5F9F9E5E9F
S31508006B505A9A9B5B99595898884849894B8B8A4A0F
S31508006B604E8E8F4F8D4D4C8C44848545874746867F
S31508006B708242438341818040986B0008C800002008
S31508006B8004010000504600089C6C0008CC01002057
S31508006B903C080000604600080000000000000000F5
S31508006BA000000000000000000000000000000000D7
S31508006BB000000000000000000000000000000000C7
S31508006BC000000000000000000000000000000000B7
S31508006BD001020304010203040607080900A24A0485
S31508006BE0000000000000000001020304060708096F
S31508006BF00000000000000000000000000000000087
S31508006C000000000004000000010000000000000071
S31508006C100000000000000000000000000000000066
S31508006C200000000000000000000000000000000056
S31508006C300000000000000000000000000000000046
S31508006C400000000000000000000000011058594C28
S31508006C504C303131327878787878787878CB7E000D
S31508006C60011058594C4C3031313278787878787828
S31508006C70787804013205054C4C30313106145941F7
S31508006C8032303035323848343530343241787878D5
S31108006C9078787D5D7E00000000000000A2
S705080018C515
